:020000040000FA
:100000000000052800000000090083120313850189
:100010008601870183160030850086008700063040
:100020009F00851405160D168312A00117220C25BA
:100030006E260030F1000F237208F800851C34286A
:1000400003220321851C342803225E23851C3428C7
:10005000032271200511851C342803228321851C6D
:100060003428032259221E283720B6262B280515AE
:1000700001304B200511003A031D080021088400BF
:100080002A08800021084F3C031D49283030A10078
:100090000800A10A0800272202302722AA01031023
:1000A0000830AF00A0131010851870280000000061
:1000B00059281B3027221930272200000000031086
:1000C000AA0C851C6528803066280030AA07AF0B73
:1000D00059281B3027221A302722000085180034A7
:1000E0000134A01E0800A01F0800A0130515220857
:1000F000A5002808A600220884000008AB00D12033
:10010000003A031DBB2822088400003000002208AA
:100110006F3C03198E280000A20A91285030A200DB
:100120000000A80B7B28A012250884009A28A50AA5
:10013000250884000008A800210884002808800001
:1001400021084F3C031DA7283030A100A828A10A90
:100150000130AD0200002508840000308000A60BAD
:10016000B228BA2825086F3C031D97285030A500F7
:1001700084009A28080005149010101690168E011D
:100180008F0110142508A2002608A8000F08023CC1
:10019000031DC6280E08313C031DCA281010051087
:1001A000080005141B302722851801341A30272235
:1001B00000000830AF002B18EB2805141B30272255
:1001C0008518013419302722000000000310AB0C01
:1001D000AF0BDB28F92805101B302722851C0134C2
:1001E00019302722000000000310AB0CAF0BDB28F6
:1001F000F9280000051018302722851C0134000062
:10020000163027220034A01A08002030A700220848
:100210008400851C0800801B182904086F3C031902
:100220001329840A152950308400A70B09290800D6
:100230000408A200001B2429801A21290230A800EA
:1002400036290430A8003629801A29290630A8004A
:10025000362904086F3C03194C29840A0008A800B9
:10026000A80803194B29E039031D4829851C0800FB
:100270002808AF006221003E03190800851C080011
:100280002808AF00AF034F2103194A29851C080035
:1002900074210800A0160800503084002E2922087E
:1002A00084000008AB0004086F3C03195F29840A2E
:1002B0000008AB06AF0B53292B08FF3A080050305B
:1002C000840058292208840023080402031D692998
:1002D000003404086F3C03197129840AAF0B6429A8
:1002E0000134503084006E292208840000308000E0
:1002F00004086F3C03198029A20A0030A8000800F6
:100300005030A2007D29201A08002030A7002408C0
:100310008400851C0800801B982904084F3C0319A1
:100320009329840A952930308400A70B8929080075
:100330000408A400001BA429801AA1290230A900E6
:10034000B6290430A900B629801AA9290630A900C7
:10035000B62904084F3C0319CC29840A0008A900D7
:10036000A9080319CB29E039031DC829851C0800F9
:100370002908AF00E221003E03190800851C08008F
:100380002908AF00AF03CF210319CA29851C080033
:10039000F42108002016080030308400AE2924081B
:1003A00084000008AC0004084F3C0319DF29840ACC
:1003B0000008AC06AF0BD3292C08FF3A08003030F8
:1003C0008400D8292408840021080402031DE92997
:1003D000003404084F3C0319F129840AAF0BE429C7
:1003E000013430308400EE2924088400003080007D
:1003F00004084F3C0319002AA40A0030A900080091
:100400003030A400FD29A01B0800101C0922102276
:1004100008009010101690168E018F01101408001D
:100420000F08063C031D08001010A017080000303C
:10043000AD005030A300A2003030A100A400840021
:10044000800104086F3C03190800840A202A2C222A
:10045000000011302C220800AE00AE0B2D2A08003F
:1004600023086F3C031D382A5030A3008400080085
:10047000A30A840A080024084F3C031D432A303095
:10048000A40084000800A40A840A080004084F3C61
:10049000031D4D2A303084000800840A0800250816
:1004A000A400840000308000A90B572A08003B22DA
:1004B000522A201E872A24088400A5000008F6007E
:1004C000B23C031D652A0824852A0008B03C031DA0
:1004D0006B2A3124852A0008E53C031D7F2A462229
:1004E000462246220130F1000F2300087202031D4C
:1004F000882A46220008013C03191C23852A00088B
:10050000833C031D852ADB24852A4F222012080004
:100510000008031D852A46227D2AF301F901FA010C
:1005200023088400E5308000F3063022103080007C
:10053000F30630227208F4000130F1000F23720834
:100540008000F3067408F200302250308000F30679
:10055000302201308000F30630227908043E80000A
:10056000F306302276088000F306302277088000F8
:10057000F306302207308000F3063022003080007E
:10058000F30630227A08FB1B013EFC1B023EFD1BDA
:10059000043EFE1B083E8000F3063022FB137B085E
:1005A0008000F3063022FC137C088000F306302222
:1005B000FD137D088000F3063022FE137E088000C4
:1005C000F3063022F3097308800030220800710816
:1005D000031783128D00031383127208031783120B
:1005E0008C0083168C130C150B178B1355308D0054
:1005F000AA308D008C148B1363000C11031383122B
:100600000D120B138B130408F4007208F500781810
:100610000A2B0C25740884007508F2000800710884
:10062000031783128D0083168C130C1483120C088D
:1006300003138312F200080046220008F900462244
:100640000008F600013C031D332B46220008F7008A
:10065000F100462246220008F919803EF200E72206
:10066000FE008D225D2B0008023C031D462B462216
:100670000008F700FB01F1000F23FC00F10A0F2333
:10068000FD00F10A0F23FE008D225D2B0008033CC4
:10069000031D502B46220008F700D4258D225D2B28
:1006A0000008043C031D5D2B46220008F7008F253F
:1006B000A725B925CA258D225D2B0800A01A0800A0
:1006C0008316A0308400B0000330B10083120030E4
:1006D000861B013EB723851C0800061B013EB7237D
:1006E000851C0800861A013EB723851C0800061ADF
:1006F000013EB723851C08000619013EB723851C5F
:1007000008008618013EB723851C08000618013E24
:10071000B723851C0800871B013EB723851C0800F2
:10072000071B013EB723851C0800871A013EB7232B
:10073000851C0800071A013EB723851C080087198D
:10074000013EB723851C08000719013EB723851C0D
:1007500008008718013EB723851C08000718013ED2
:10076000B723851C0800851A013EB72308008316AD
:10077000801BD52B801ADD2B013C031DC02BC72B02
:1007800008300005031DC52BCD2BE923D52B0830E0
:100790000005031DCD2BE923D52B08308006F8304A
:1007A0008005D52BF0308005D52B840AB00AB10A1C
:1007B000B10AB10A831200300800001FE42B013C8B
:1007C000031DCF2BE923D52B003C031DCF2BE923A1
:1007D000D52B07300005073C031DEF2B072C0330FA
:1007E0000005033C031D062C0008B200321EF92B45
:1007F000FB2B3216FC2B32123208800083124E255E
:1008000083163008840007308004072C800A080013
:100810003B2200088316BE0083123B220008831689
:10082000BF00A030BD00C030840000083E02031DA0
:10083000272C840A00083F02031D202C9B24282C0F
:100840000008103E3F02031D282C5E24282C840A39
:10085000840ABD0A0408E03C031D152C2F2C8312CA
:1008600008003B2200088316BE0083123B220008CA
:100870008316BF00A030BD00C030840000083E02D7
:10088000031D522C840A00083F02031D492C5E24DC
:10089000532C0008801A5C2C203E3F02031D532C71
:1008A0009B24532C840A840ABD0A0408E03C031DDF
:1008B0003E2C5A2C83120800E03E4D2C0408B20056
:1008C0003D088400001F702C692C831632088400B8
:1008D000D82C8312F61C652C831632088400742CE5
:1008E0008312F61C6C2C652C3D080F39B2003207C0
:1008F0000A15831282078617D82C0617D82C86165D
:10090000D82C0616D82C0615D82C8614D82C0614EC
:10091000D82C8717D82C0717D82C8716D82C071651
:10092000D82C8715D82C0715D82C8714D82C071449
:10093000D82C8516D82C0408B2003D088400001F6E
:10094000AD2CA62C831632088400D82C8312F61CFA
:10095000A22C831632088400B12C8312F61CA92C19
:10096000A22C3D080F39B20032070A158312820704
:100970008613D82C0613D82C8612D82C0612D82C05
:100980000611D82C8610D82C0610D82C8713D82CFA
:100990000713D82C8712D82C0712D82C8711D82CE3
:1009A0000711D82C8710D82C0710D82C8512D82CDA
:1009B00083160A1108008316A0308400F830000561
:1009C000801A103A8000840A0408A43C0319E92C18
:1009D000DE2CF9300005801A103A8000840A0408E1
:1009E000A83C0319F42CE92CFA300005801A103ABF
:1009F0008000840A0408AC3C0319FF2CF42CFB3063
:100A00000005801A103A8000840A0408B03C0319DB
:100A10000A2DFF2C8312080083160330B000A0308B
:100A2000840030088312F1000F23720883168000BF
:100A3000840AB00AB00AB00A0408B03C031D112DA4
:100A40000330B000C030840030088312F1000F235F
:100A500072088316B200B21B352D8000840A800014
:100A6000840AB00AB00AB00A482DB00A30088312CE
:100A7000F1000F23720883168000840AB00A300840
:100A80008312F1000F23720883168000840AB00AD3
:100A90000408E03C031D242D831208008316B10ACC
:100AA00031088312F1000F23F30123088400B230D0
:100AB000F21FB0308000F30630227610F21B76145D
:100AC000F21372088000F30630228316B10A31084F
:100AD0008312F1000F23F21372088316B21A7F2DCE
:100AE000B21D732D812D8312761C772D792D203E1A
:100AF000812D781D7D2DF03E812D103E812D321AE5
:100B0000203E83127F398000F3063022F3097308F8
:100B1000800030228316B103B103831208008316CC
:100B200006088312FB000739FC00FC0D7B08F03936
:100B3000FB007C08FB078316070883128039031D1E
:100B4000A22DA42D7B14A52D7B10FB09080000000D
:100B50000608FC000739FD00FD0D7C08F039FC009B
:100B60007D08FC07871FB52DB72D7C10B82D7C1490
:100B70000800831607088312FD00FD0D8316050883
:100B800083122039031DC52DC72D7D14C82D7D105E
:100B9000FD0908000708FE00FE0D851ED02DD22D90
:100BA0007E10D32D7E1408004622462246220008DD
:100BB000FA0046220008FB007A18FB1746220008BC
:100BC000FC00FA18FC1746220008FD007A19FD17F0
:100BD00046220008FE00FA19FE17FB1FF52DFC1F28
:100BE000F22DF42D8613F52D86177B1FFD2D7C1F0E
:100BF000FA2DFC2D0613FD2D0617FB1E052EFC1EDF
:100C0000022E042E8612052E86167B1E0D2E7C1EAD
:100C10000A2E0C2E06120D2E0616FB1D152EFC1D7F
:100C2000122E142E0611152E06157B1D1D2E7C1D51
:100C30001A2E1C2E86101D2E8614FB1C252EFC1C25
:100C4000222E242E0610252E06147B1C2D2E7C1CF5
:100C50002A2E2C2E87132D2E8717FD1F352EFE1FB3
:100C6000322E342E0713352E07177D1F3D2E7E1F83
:100C70003A2E3C2E87123D2E8716FD1E452EFE1E57
:100C8000422E442E0712452E07167D1E4D2E7E1E27
:100C90004A2E4C2E87114D2E8715FD1D552EFE1DFB
:100CA000522E542E0711552E07157D1D5D2E7E1DCB
:100CB0005A2E5C2E87105D2E8714FD1C652EFE1C9F
:100CC000622E642E0710652E07147D1C6D2E7E1C6F
:100CD0006A2E6C2E85126D2E851608008316003044
:100CE000860087008512A0308400801B782E86172E
:100CF000840A801B7C2E0617840A801B802E861691
:100D0000840A801B842E0616840A801B882E0615F2
:100D1000840A801B8C2E8614840A801B902E061455
:100D2000840A801B942E8717840A801B982E07172D
:100D3000840A801B9C2E8716840A801BA02E07160F
:100D4000840A801BA42E8715840A801BA82E0715F1
:100D5000840A801BAC2E8714840A801BB02E0714D3
:100D6000840A801BB42E85168312080012302C22B0
:100D7000851C080012302C22851C080012302C2201
:100D8000851C080012302C22851C080012302C22F1
:100D9000851C080012302C22851C080012302C22E1
:100DA000851C080012302C22851C080012302C22D1
:0E0DB000851C080012302C22851C080008004B
:084000000100030005000000AF
:02400E00F23F7F
:10420000000051000100800000000000800000005C
:104210000000C00004002000C00004000000800076
:10422000000000008000000000008000000000008E
:10423000800000000000800000000000C0000500B9
:104240002000C000050000002F001C0010000F001F
:104250001D00100080000000000080000000000031
:064260000F0084001000B5
:00000001FF
